:100000001C308A00B12C0000491943104529D22721
:10001000520020102010201020102010201020103E
:10002000201000012010201020102010201020107F
:10003000201020100000A0183617300032192E189A
:100040003500A01932173000201A34173100201A59
:1000500038173000201B34173000201C38173200AE
:10006000A01C36173000311938173000B11B361775
:100070003400B11C32173000B21A36173000B31AF0
:1000800032173800331C3417300020193417300071
:100090006B247A100001A02AEE35EE377737200066
:1000A000A0183019B435483D2000A018B418B13557
:1000B000483D20002019301AB835483D200020194D
:1000C0003819B235483D2000A019B01BB235483D63
:1000D0002000201AB01CB635483D2000A01A361A60
:1000E000B535483D2000201B311AB435483D20006D
:1000F000201CB11CB235483D2000B1182E19B9267C
:10010000483D200031192E19B926483D2000311BE9
:10011000AE19B826483D20003219AE1AB826483D1F
:100120002000321AAE1AB826483D2000A018B51992
:10013000B635483D2000A02AEE35EE37773720004F
:100140002010D020D220CD22D42252102000201006
:100150004927492AC920CC24DA222000CC27C325EC
:10016000AD204C002025C31655274C00C420C316D3
:1001700055274C00CC27C325AD274B002010CE3788
:10018000A020542A0001AE1A642100012E18642117
:1001900000005328C424C618201000015328C4248A
:1001A0004619201000015328C424C619201000014C
:1001B0005328C424461A20100001D021CD16491915
:1001C00053100001D021CD16522520100001C42962
:1001D000C416492720100001D316C429441020104A
:1001E00000005328C424C618201000015328C4243A
:1001F0004619201000015328C424C61920100001FC
:100200005328C424461A20100001D021CD164927B6
:1002100020100001C429C416492720100001D3165C
:10022000C4294410201000015328C424C6185010BB
:1002300000015328C4244619501000015328C42437
:10024000C619501000015328C424461A501000014A
:10025000492754104529521000004D18A518641064
:1002600044284C262D262027D526201000004D1886
:10027000A518641044284C262D292027D5262010A7
:1002800000004D18A5186410202250264C10C220E2
:100290004E22AD2B0001C232733A20102010000113
:1002A000CE372010201020100001CC37F732733ADF
:1002B00020100001CC377710201020100001CD3223
:1002C000E416CC3777100001CD32E434F536201037
:1002D0000001CD326424E93368100001C83467346A
:1002E000201020100001C8346734E5397410000074
:1002F0004D18A5186410A0265526DF2943264B105B
:100300002010200041264C104F2346102000532877
:10031000C424461020102000D0214D16C4294410BA
:10032000200041264C104F27201020004D18A51802
:100330006410CA2120216137E42B69327434000132
:10034000CC27D722532A20102000CC27571020106A
:1003500020102000CD244410201020102000CD2497
:10036000C416C82447242000C82447242010201085
:1003700020004D18A5186410C6244C2A4529A02930
:1003800045262E10000120102010C620532A2029B7
:100390006F36EC3766330001201020105326CF2B28
:1003A00020296F36EC37663300004D18A51864100D
:1003B000D332F23461362021693A731000012010E3
:1003C000201020002021693A7310201020004D18C1
:1003D000A5186410D332F234613620234D2A201040
:1003E0000001A024B22920234F29CD205410201031
:1003F000201000012026653374102025F539F434CF
:10040000E634653200012029E933683A2025F539C0
:10041000F434E634653200004D18A5186410D03766
:10042000EC30F234F43CA039653A00012010A020F1
:100430006E3AE9165034E1396510201000012010A1
:100440002010A024EE165034E13965102010000071
:10045000CD12323220105034E1396510F33274106D
:10046000201000012010A0206E3AE9165034E13926
:1004700065102010000120102010A024EE1650342A
:10048000E139651020100000CD123232A024492934
:100490002021AD2B69327434000120102010CE379A
:1004A000F23661362010201020100001201020109C
:1004B00035186B14E432E6307536F4140001201060
:1004C000201036186B102010201020102010000172
:1004D0002010201037186B10201020102010201032
:1004E0000000CD1232322010CF294610C23CF0302D
:1004F000F339200020224929C52154106639EF36EE
:10050000A024B2290001A02AD322A027532320230C
:100510004926D42252100000CD1232322010CD2AAA
:100520004C1031193810532A2000202250264C102C
:10053000D3225410C22CA018321C000120274F29AE
:10054000CD204C1044284C26A029452A0000CD126D
:1005500032322010CA34743A6539202965322E00AF
:10056000D52945104A2920100001C23CF030F3394A
:1005700020100000CD123232A028D5204E2A492D5D
:100580004529201020002010201B2D21693A7314CA
:10059000E4326617291000012010A01B2D21693AB2
:1005A000731020102010201000012010201C2D217D
:1005B000693A731020102010201000012010A01C98
:1005C0002D21693A731020102010201000012010F6
:1005D0002010D732EC31EF36203A6F102010000196
:1005E00020234622C1213918311C4410F61861100D
:1005F000000120102022C1213918311C4410F618A6
:10060000611000004B308400831300080319162B7F
:100610000330F800F701F70B0B2BF80B0A2B3C30DB
:10062000F700F70B112B142B800B082B08008714F5
:10063000192B1A2B000007112011200883168700A0
:10064000212B222B000083128710262B272B000042
:10065000080020152008831687002E2B2F2B000062
:1006600083128714332B342B00008710372B382B41
:100670000000080007112011200883168700402B76
:10068000412B000083128714452B462B0000871056
:10069000492B4A2B00000800CA014A08063C031CEB
:1006A0005A2BC91F552B2923562B3A230310C90D4A
:1006B000CA0A4D2B0800511E5F2B8516602B851230
:1006C000D11D642B0617652B0613511D692B861748
:1006D0006A2B8613D11C6E2B06166F2B0612511C2B
:1006E000732B8616742B861208000516772B0512BD
:1006F000792B08004B08003A0319882B013A03199B
:10070000892B033A03198C2B013A03198F2B922B57
:10071000932B4030CA07932B1430CA07932B5430C5
:10072000CA07932B932B80304A07CD004D08CE008B
:100730004E0EF7000F30F70577080F39D0004E083E
:100740000F39CF005008D1005B2375232130F7000B
:10075000F70BA82B4F08D1005B2375232130F7003E
:10076000F70BB02B08004D0ECE000F30CE05CD0597
:1007700010304E07CF00D1005B23752310304D079A
:10078000CF00D1005B2375232130F700F70BC62B78
:100790000800831603178C170C1400000000831246
:1007A0000C087F3903190D2C0313CA0003170D0819
:1007B0000313CB0003170F080313CC004A08CD0026
:1007C000B3234B0803178D0003134C0803178F0046
:1007D00083168C170C140000000083120C0D0E0DF4
:1007E0007F3903190D2C0313CA0003170D080313D7
:1007F000CB0003170F080313CC004A08CD00B32326
:100800004B0803178D0003134C0803178F008D0A44
:1008100003198F0A0313C92B031703130800C90117
:100820002015200883168700152C162C0000831233
:1008300087141A2C1B2C0000071D272C1F2C202C82
:100840000000C90A4908643C0319272C1C2C871096
:10085000292C2A2C00002C2C2D2C000007112011F3
:10086000200883168700342C352C00008312490899
:10087000643C031D502CCA01CB017A2304300317BA
:100880008D0000308F000313C9230430CA00FA30F2
:10089000CB000223CA0B472C0130F800532C532CF9
:1008A0000030F800532C080007112011200883168F
:1008B00087005A2C5B2C0000831287145F2C602C5D
:1008C00000002015200883168700662C672C000086
:1008D0008312080017234508C9004C233A230F242C
:1008E000F8080319772C54240130F800A62CC8010D
:1008F0004808073C031C852CC61F802C2923812C0B
:100900003A230310C60DC80A782C0F24F8080319DF
:100910008D2C54240130F800A62CC8014808073C4F
:10092000031C9B2CC71F962C2923972C3A230310BA
:10093000C70DC80A8E2C0F24F8080319A32C5424C1
:100940000130F800A62C54240030F80008002030B4
:10095000C5003E08C6003F08C7006A2408001723E8
:100960004308C9004C233A230F24F8080319BC2C70
:1009700054240130F8002C2DC5014508073C031C08
:10098000CA2CC41FC52C2923C62C3A230310C40D1E
:10099000C50ABD2C8714CC2CCD2C000020152008B6
:1009A00083168700D32CD42C000083128710D82CF8
:1009B000D92C00008714DC2CDD2C0000071120113D
:1009C000200883168700E42CE52C00008312871092
:1009D000E92CEA2C00004308C9004C2329230F24EA
:1009E000F8080319F72C54240130F8002C2DC60107
:1009F000C5014508073C031C192D0310C60D201521
:100A000020088316870083128714062D072D000007
:100A1000071D0D2D0130C7000E2DC7018710102DA9
:100A2000112D00004708F800F808031D4614C50AF8
:100A3000F92C20152008831687001E2D1F2D00007D
:100A400083128714232D242D00008710272D282D95
:100A5000000054244608F80008000730BB053B0896
:100A6000BD00BD0DBD0DBD0DF830BD053830BD0557
:100A70003B08BD042030C3000430C400AF24780814
:100A8000BC00C030BC053D08BC040430BE003C08BE
:100A9000BF00A724080083168512051286120612CD
:100AA000861306138312A010200883168700831272
:100AB0008714201220088316870083120712A011C2
:100AC000200883168700831287151F139F1783162C
:100AD0009F1783121F14831603170908C039890052
:100AE00003131F129F120130031788000030F80013
:100AF000831203131F08C33978049F000730900046
:100B0000FF30831695008113831207160A30CB003D
:100B10000223E830C5000630C600FF30C7006A2453
:100B2000E830C5000330C600FF30C7006A24E83053
:100B3000C5000730C600AF30C7006A24EA30C500E0
:100B40000630C6000F30C7006A24EA30C500033003
:100B5000C600FF30C7006A24EA30C5000730C6006F
:100B6000C7016A24BE01BF01A7240130BE000230C4
:100B7000BF00A7240230BE00BF01A7240330BE007F
:100B8000B030BF00A7240430BE009830BF00A724B7
:100B90000530BE008830BF00A7240630BE007F307D
:100BA000BF00A724BB012D258A150A16F22C64303C
:100BB000CB0002230330D1005B2375230530CB002B
:100BC00002230330D1005B2375230130CB000223C5
:100BD0000330D1005B2375230130CB0002230230A8
:100BE000D1005B2375230130CB0002230230D100FA
:100BF0005B2375230130CB0002230E30D1005B2331
:100C000075230130CB000223D1015B237523013012
:100C1000CB0002230830D1005B2375230130CB00C9
:100C20000223D1015B2375230130CB0002230C305A
:100C3000D1005B2375230130CB000223D1015B235C
:100C400075230130CB0002230630D1005B237523CE
:100C50000130CB000223D1015B2375230130CB008F
:100C600002230130D1005B2375230230CB00022325
:100C70008A150A16F72CD1015B2375230230D100A7
:100C80005B2375230230CB0002238A150A16FC2C45
:100C9000E830C3000330C400AF247808BC00E8305B
:100CA000C3000730C400AF247808BB00BA0803199A
:100CB0005E2ECF30BB053C12BC16602E3030BB041C
:100CC000E830C5000330C6003C08C7006A24E8309D
:100CD000C5000730C6003B08C7006A2408009030F2
:100CE000C5004308C6004408C7006A249230C50006
:100CF0004308C6004408C7006A2408003D08BF0036
:100D00003C08BE003D08013C031C942E031D8C2EA4
:100D10003C08003C031C942E03103D0CFA003C0CD4
:100D2000F900FF3CC000C92E3D08023C031CB32E55
:100D3000031D9E2E3C08003C031CB32E00303C02D9
:100D4000C3003D08C4000130031C0230C402440C3F
:100D5000FA00430CF900FA0CF90C3F30FA05790857
:100D6000803CC000C92EFE303C02C3003D08C400D8
:100D70000130031C0230C402440CFA00430CF90099
:100D8000FA0CF90CFA0CF90C1F30FA057908403C02
:100D9000C0009030C300C401AF247808C2004008EE
:100DA00042020319832FC1014108073C031CDF2EB7
:100DB0004108C3004008C4006F26C10AD42E3F0872
:100DC000C4003E08C3004408C9004308C800CB0162
:100DD0002830CA001030CC00F701FA01C90CC80C49
:100DE000031CF82E4A08F7070318FA0A4B08FA07FB
:100DF000FA0CF70CF90CF80CCC0BEE2E7908C600A7
:100E00007808C5004608C500C6010310C60CC50C0D
:100E1000C408031D122F4308043C031C122FC601F3
:100E2000C501162F0130C5070318C60AC608031DE1
:100E30001D2F45084F3C0318202FC6015030C50018
:100E40004508C7004708C80005112930F700F70B0F
:100E5000272F0000481C2E2F05152F2F0511293094
:100E6000F700F70B312F0000C81C382F0515392F5C
:100E700005112930F700F70B3B2F0000481D422FCA
:100E80000515432F05112930F700F70B452F0000FA
:100E9000C81D4C2F05154D2F05112930F700F70BF4
:100EA0004F2F0000481E562F0515572F05112930CA
:100EB000F700F70B592F0000C81E602F0515612F92
:100EC00005112930F700F70B632F0000481F6A2F28
:100ED00005156B2F05112930F700F70B6D2F00005A
:100EE000C81F742F0515752F05112930F700F70B52
:100EF000772F000005152930F700F70B7D2F000034
:100F00000130CB0002234008A1000800CA01CB0138
:100F10007A230800CA010130CB007A230800EA30A6
:100F2000C3000230C400AF247808BD00BB08031919
:100F30009B2FBD139C2FBD17EA30C5000230C600A1
:100F40003D08C7006A2408009030C3000830C40080
:100F5000AF247808BC00BB080319B02FBC17B12F11
:100F6000BC130830C3003C08C4006F2608004208C8
:100F7000F80141020318BF2F4108F700CB2FF701FA
:100F80000830C300C10DF70D420877020318F700BF
:100F9000F80DC30BC22F0800BB01071BBB16871B34
:100FA0003B16E830C3000130C400AF247808BC0011
:100FB000BC18BB153C183B15BC1B3B14E830C300E8
:100FC000C401AF247808BD003D1BBB143B08F800EA
:100FD00008009030C3003908C400AF247808BA0074
:0E0FE000BB003730BC008A153B278A11080081
:10100000BB01BA01BC013C080F3C031C29289F14FA
:101010003D109F1C3D143D1811283D109F1C3D1490
:101020000B289F1811281E08FA0083161E08831229
:10103000BE001E08BF003E08F8003F08F90079080E
:10104000FA007808BA0779080318790FBB07BC0AB9
:101050000328BB0CBA0CBB0CBA0CBB0CBA0CBB0CF7
:10106000BA0C0F30BB052D0B63282C083B02031C68
:101070004728031D3F283A082B02031847283B083E
:10108000AC003A08AB00F8002C08F90095280130B4
:101090003A07F8003B08FA000318FA0A7A082C020B
:1010A000031C6228031D58282B08780203186228A5
:1010B0003B08AC003A08AB00AD012B08F8002C0847
:1010C000F900952891283B082C02031C7528031D64
:1010D0006D282B083A02031875283B08AC003A0823
:1010E000AB00F8002C08F900952801302B07BD0053
:1010F0002C08BE000318BE0A3E083B02031C9128C0
:10110000031D86283A083D02031891283B08AC00CD
:101110003A08AB000130AD002B08F8002C08F900AC
:1011200095282B08F8002C08F900080003178D01FA
:1011300083168C130C1483120C080313A200061CD4
:10114000A72822080A3C031CA728220F64298A1119
:1011500086278A15093003178D0000308F008A1109
:101160000313C9238A158A118A278A151230031797
:101170008D0000308F008A110313C9238A158A114C
:1011800086278A15A03003178D0000308F008A1142
:101190000313C9238A158A118A278A15A7300317D2
:1011A0008D0000308F008A110313C9238A1508307F
:1011B000B6003608193C031C05299030C3003608D8
:1011C000C4008A11AF248A157808BA0036080317BC
:1011D0008D0003133A0803178C0083168C130C152B
:1011E000831203130B08F7008B1383160317553074
:1011F0008D00AA308D008C148C18FC280C117708F7
:10120000831203138B04B60AD928A20103178D0198
:101210000313220803178C0083168C130C158312FA
:1012200003130B08F7008B138316031755308D003B
:10123000AA308D008C148C181B290C11770883128E
:1012400003138B04A501013003178D000313250838
:1012500003178C0083168C130C15831203130B08D1
:10126000F7008B138316031755308D00AA308D00BD
:101270008C148C1839290C117708831203138B04F2
:101280000430A600023003178D000313260803174D
:101290008C0083168C130C15831203130B08F700B4
:1012A0008B138316031755308D00AA308D008C14D4
:1012B0008C1858290C117708831203138B0464309F
:1012C000CB008A1102238A150830B6003608193C73
:1012D000031C9B29360803178D0083168C130C14EE
:1012E00083120C080313B7003608113C0319802938
:1012F0003608C3003708C4008A116F268A15992959
:1013000037087F39B900391437088138B800903070
:10131000C5003608C6003908C7008A116A248A1534
:101320009230C5003608C6003808C7008A116A2402
:101330008A15B60A662903178D0183168C130C14BF
:1013400083120C080313A200013003178D008316CB
:101350008C130C1483120C080313A500023003171E
:101360008D0083168C130C1483120C080313A60033
:101370008A150A166C2D2208003A0319DE29013A53
:101380000319DE29033A0319DE29013A0319DE297C
:10139000073A0319F629013A0319092A033A0319EE
:1013A0001C2A013A03192F2A0F3A03192F2A013A4E
:1013B00003192F2A033A03192F2A482ABB018A113D
:1013C0008F278A15EA30C5000330C600BD30C7003C
:1013D0008A116A248A152208BB008A112D258A15D4
:1013E0000130BB008A11A4278A15492A0130BB00AD
:1013F0008A118F278A15EA30C5000330C60077307E
:10140000C7008A116A248A15BB018A11A4278A158C
:10141000492A0130BB008A118F278A15BB018A1126
:10142000A4278A15EA30C5000330C600EE30C70095
:101430008A116A248A15492A0130BB008A118F2734
:101440008A15BB018A11A4278A15EA30C50003302A
:10145000C600DB30C7008A116A248A15492ABB01FD
:101460008A118F278A15EA30C5000330C60077300D
:10147000C7008A116A248A1507302202B900BB000E
:101480008A112D258A15BB018A11A4278A15492A9C
:10149000492A080020303C1E3030BD003B08F700D0
:1014A000BB1F592AF709F70A7708BB002D30BD008A
:1014B000BC173B08C1006430C2008A11B7278A15E7
:1014C0007708BB0030307807BE003B08C1000A3007
:1014D000C2008A11B7278A1530307707C000303034
:1014E0007807BF003D08F700BC1D782ABC1F3C11DF
:1014F0003C1A852ABC1FA02A3C19A02A7708BE00E6
:10150000BC18A02A7708BF00A02A30303E02031D75
:10151000A02A7708BE002030BD00BC1D932A3C11D4
:10152000BC14BC1FBC1030303F02031DA02A77083A
:10153000BF002030BE00BC1D932ABC10BC1F3C1055
:101540003C1DA72A3D08CD008A11B3238A15BC1C77
:10155000AE2A3E08CD008A11B3238A153C1CB52A59
:101560003F08CD008A11B3238A154008CD008A11A7
:10157000B3238A150800A108031DC72ABE3003172C
:101580008D0000308F008A110313C9238A152108AA
:10159000C73C0318D92A0310210CBA002D30CD0006
:1015A0008A11B3238A153A08BB001330BC004A22C3
:1015B000072B2108133C0318F02A0310210CBA0052
:1015C0002030CD008A11B3238A152D30CD008A1129
:1015D000B3238A153A08BB001130BC004A22072BFE
:1015E0000310210CBA002030CD008A11B3238A15D4
:1015F0002030CD008A11B3238A152D30CD008A11F9
:10160000B3238A153A08BB001830BC004A22211CBB
:10161000132BC33003178D0000308F008A11031382
:10162000C9238A151C2BC63003178D0000308F008C
:101630008A110313C9238A1508008F018E010A300D
:10164000CB008A1102238A150F08FA000E08F70052
:101650000F087A02031D242B7708BB007A08BC0010
:10166000BD01BC08031D382B3B089D3C0318422BD1
:10167000BC08031D422B3B08A23C031C422B01303B
:10168000BD00832CBC08031D492B3B08D93C031823
:10169000532BBC08031D532B3B08DF3C031C532B6F
:1016A0000230BD00832C3C08003C03186B2BFF3A32
:1016B000031D5E2B3B083B3C03186B2B3C08013C95
:1016C000031C6B2B031D682B3B08443C031C6B2B3A
:1016D0000330BD00832C3C08003C0318832BFF3AE9
:1016E000031D762B3B08B33C0318832B3C08013CBD
:1016F000031C832B031D802B3B08BE3C031C832B48
:101700000430BD00832C3C08003C03189B2BFF3A9F
:10171000031D8E2B3B08DA3C03189B2B3C08013C35
:10172000031C9B2B031D982B3B08E53C031C9B2BA8
:101730000530BD00832C3C08013C0318B32BFF3A55
:10174000031DA62B3B08783C0318B32B3C08023C36
:10175000031CB32B031DB02B3B08873C031CB32B8E
:101760000630BD00832C3C08023C0318CB2BFF3A0B
:10177000031DBE2B3B08683C0318CB2B3C08033CE5
:10178000031CCB2B031DC82B3B087B3C031CCB2B22
:101790000730BD00832C3C08023C0318E32BFF3AC2
:1017A000031DD62B3B08B53C0318E32B3C08033C38
:1017B000031CE32B031DE02B3B08CA3C031CE32B5B
:1017C0000830BD00832C3C08033C0318FB2BFF3A78
:1017D000031DEE2B3B08F23C0318FB2B3C08053C99
:1017E000031CFB2B031DF82B3B080D3C031CFB2BA0
:1017F0000930BD00832C3C08053C0318132CFF3A2C
:10180000031D062C3B08D13C0318132C3C08063C56
:10181000031C132C031D102C3B08F63C031C132C3B
:101820000A30BD00832C3C08063C03182B2CFF3AE1
:10183000031D1E2C3B086B3C03182B2C3C08073C5B
:10184000031C2B2C031D282C3B08943C031C2B2C25
:101850000B30BD00832C3C08083C0318432CFF3A96
:10186000031D362C3B08E53C0318432C3C080A3C7E
:10187000031C432C031D402C3B081A3C031C432C27
:101880000C30BD00832C3C080C3C03185B2CFF3A49
:10189000031D4E2C3B08AB3C03185B2C3C080D3C55
:1018A000031C5B2C031D582C3B08DE3C031C5B2CEB
:1018B0000D30BD00832C3C080D3C0318732CFF3AFF
:1018C000031D662C3B08D83C0318732C3C080F3CC6
:1018D000031C732C031D702C3B08273C031C732C2A
:1018E0000E30BD00832CBC08031D7A2C3B08EC3C59
:1018F0000318832CBC08031D832C3B08F33C031CFA
:10190000832C0F30BD003D08F80008001D23780827
:10191000BA003A08003C0318612D3A080F3C031C3A
:10192000612D3A08013A0319C02C033A0319CA2C55
:10193000013A0319D42C073A0319DE2C013A031992
:10194000E82C033A0319F22C013A0319FC2C0F3A44
:101950000319062D013A0319102D033A03191A2D04
:10196000013A0319242D073A03192E2D013A0319C0
:10197000382D033A0319422D013A03194C2D562DE7
:101980001B3003178D0000308F008A110313C92309
:101990008A15572D1E3003178D0000308F008A11D5
:1019A0000313C9238A15572D213003178D000030EA
:1019B0008F008A110313C9238A15572D243003176A
:1019C0008D0000308F008A110313C9238A15572D0B
:1019D000273003178D0000308F008A110313C923AD
:1019E0008A15572D2A3003178D0000308F008A1179
:1019F0000313C9238A15572D2D3003178D0000308E
:101A00008F008A110313C9238A15572D303003170D
:101A10008D0000308F008A110313C9238A15572DBA
:101A2000333003178D0000308F008A110313C92350
:101A30008A15572D363003178D0000308F008A111C
:101A40000313C9238A15572D393003178D00003031
:101A50008F008A110313C9238A15572D3C300317B1
:101A60008D0000308F008A110313C9238A15572D6A
:101A70003F3003178D0000308F008A110313C923F4
:101A80008A15572D423003178D0000308F008A11C0
:101A90000313C9238A15572D453003178D000030D5
:101AA0008F008A110313C9238A15572D572D4830EB
:101AB00003178D0000308F008A110313C9238A1584
:101AC0006A2D4B3003178D0000308F008A110313ED
:101AD000C9238A1508001D237808BA00013A0319A2
:101AE0009C2D033A0319A62D013A0319B02D073A8C
:101AF0000319BA2D013A0319C42D033A0319CE2D47
:101B0000013A0319D82D0F3A0319E22D013A0319AE
:101B1000EC2D033A0319F62D013A0319002E073A6A
:101B200003190A2E013A0319142E033A03191E2E23
:101B3000013A0319282E322E503003178D00003041
:101B40008F008A110313C9238A153C2E55300317C1
:101B50008D0000308F008A110313C9238A153C2E93
:101B60005A3003178D0000308F008A110313C923E8
:101B70008A153C2E5F3003178D0000308F008A11CC
:101B80000313C9238A153C2E643003178D000030DF
:101B90008F008A110313C9238A153C2E693003175D
:101BA0008D0000308F008A110313C9238A153C2E43
:101BB0006E3003178D0000308F008A110313C92384
:101BC0008A153C2E733003178D0000308F008A1168
:101BD0000313C9238A153C2E783003178D0000307B
:101BE0008F008A110313C9238A153C2E7D300317F9
:101BF0008D0000308F008A110313C9238A153C2EF3
:101C0000823003178D0000308F008A110313C9231F
:101C10008A153C2E873003178D0000308F008A1103
:101C20000313C9238A153C2E8C3003178D00003016
:101C30008F008A110313C9238A153C2E9130031794
:101C40008D0000308F008A110313C9238A153C2EA2
:101C5000963003178D0000308F008A110313C923BB
:101C60008A153C2E9B3003178D0000308F008A119F
:101C70000313C9238A153C2E08008A11CC278A1524
:101C80007808BA000930CA000130CB008A117A23E3
:101C90008A153A082A39283C031D582EAE300317FE
:101CA0008D0000308F008A110313C9238A157F2EFF
:101CB0003A082A392A3C031D672EB23003178D00DB
:101CC00000308F008A110313C9238A157F2E3A082A
:101CD0002839283C0319762EB63003178D000030C2
:101CE0008F008A110313C9238A157F2EBA30031778
:101CF0008D0000308F008A110313C9238A15080054
:101D0000BB01BA010619BA0A3A0827020319942E30
:101D10003A08A7000A30CB008A1102238A15BA08B4
:101D2000031D942E0330BB00BA018619BA0A3A0883
:101D300028020319A72E3A08A8000A30CB008A11FE
:101D400002238A15BA08031DA72E0430BB00BA016E
:101D50000618BA0A3A0829020319BA2E3A08A90045
:101D60000A30CB008A1102238A15BA08031DBA2E45
:101D70000130BB00BA018618BA0A3A082A020319D0
:101D8000CD2E3A08AA000A30CB008A1102238A1508
:101D9000BA08031DCD2E0230BB003B08F800080036
:101DA0003A08033A0319D82E073A0319DE2EE62E15
:101DB000A40A24082302031CA401E72EA408031983
:101DC000E32EA403E52E2308A400E72EE72E080047
:101DD000831603178C170C14000000000318192F2A
:101DE00083120C087F390313BB0003170D0803137C
:101DF000BC0003170F080313BD003B08CD008A1178
:101E0000B3238A153C0803178D0003133D080317FD
:101E10008F0083168C170C1400000000831203132C
:101E2000BA0B132F162F83160317192F3A2F831669
:101E3000031783120C0D0E0D7F390313BB0003171C
:101E40000D080313BC0003170F080313BD003B0864
:101E5000CD008A11B3238A153C0803178D000313A4
:101E60003D0803178F008D0A03198F0A031003130F
:101E7000BA0BE82E0800BC1B4F2F0F30F7003B0EAB
:101E8000F7050A3077020318482F3030F7074A2F3A
:101E90003C08F7077708CD008A11B3238A150F3065
:101EA000BB050A303B020318572F3030592FBC13A3
:101EB0003C08BB073B08CD008A11B3238A150800F4
:101EC0009230C3003908C4008A11AF248A157808FB
:101ED000BA00BB003730BC003B2708008A11CC2772
:101EE0008A157808BA000830CA000130CB008A1180
:101EF0007A238A152030CD008A11B3238A15BA1EA1
:101F0000872F4C30CD008A11B3238A158C2F553082
:101F1000CD008A11B3238A15BA1D942F4C30CD0001
:101F20008A11B3238A15992F5530CD008A11B32316
:101F30008A153A1EA12F4D30CD008A11B3238A1580
:101F4000A62F2A30CD008A11B3238A153A1DAE2F51
:101F50004D30CD008A11B3238A15B32F2A30CD001E
:101F60008A11B3238A152030CD008A11B3238A1534
:101F7000BA1CC02F5530CD008A11B3238A15C52F46
:101F80004C30CD008A11B3238A153A1CCD2F2D3049
:101F9000CD008A11B3238A15D22F5330CD008A1178
:061FA000B3238A150800BE
:102000000A1286270A16360B27284D30CD000A12F1
:10201000B3230A163030CD000A12B3230A1636084D
:10202000BB001830BC000A128A154A220A168A110F
:102030002F3003178D0001308F0003140D30031370
:10204000BA000A128A15E8260A168A1148284D3065
:10205000CD000A12B3230A163030CD000A12B32382
:102060000A163608BB001830BC000A128A154A222C
:102070000A168A11393003178D0001308F000314BE
:102080000D300313BA000A128A15E8260A168A11BF
:102090000A128A270A163608B8000A128A270A1670
:1020A000380B67281F30B9000A12E9270A161E30BC
:1020B000B9000A12E9270A161D30B9000A12E927E9
:1020C0000A161C30B9000A12E9270A1683281F30A5
:1020D000B9000A128A1560270A168A111E30B90043
:1020E0000A128A1560270A168A111D30B9000A12D1
:1020F0008A1560270A168A111C30B9000A128A153F
:1021000060270A168A110A128A156E270A168A1182
:102110000A128A1580260A168A117808B70037082D
:10212000BA000A128A15D0260A168A1108009030C1
:10213000C5003A08C6003B08C7000A126A240A16FE
:102140009230C5003A08C6003B08C7000A126A244C
:102150000A163A0803178D0003133B0803178C0077
:1021600083168C130C15831203130B08F7008B13C3
:102170008316031755308D00AA308D008C148C18EF
:10218000BF280C117708831203138B0408000A126E
:1021900086270A164D30CD000A12B3230A163030B6
:1021A000CD000A12B3230A162408BB001830BC0065
:1021B0000A128A154A220A168A11433003178D0023
:1021C00001308F0003140D300313BA000A128A1570
:1021D000E8260A168A110A128A270A169030C300C6
:1021E0000B30C4000A12AF240A167808B7009030EA
:1021F000C3001930C4000A12AF240A167808B800C8
:10220000B81C0C294B3003178D0001308F000A12C7
:102210000313C9230A16772937081C3903192629FD
:10222000043A031930290C3A03193A29043A0319DC
:1022300044291C3A03194E29043A031958290C3A27
:1022400003196229043A03196C29762950300317BF
:102250008D0001308F000A120313C9230A16772953
:10226000553003178D0001308F000A120313C92364
:102270000A1677295A3003178D0001308F000A1291
:102280000313C9230A1677295F3003178D00013025
:102290008F000A120313C9230A1677296430031723
:1022A0008D0001308F000A120313C9230A16772903
:1022B000693003178D0001308F000A120313C92300
:1022C0000A1677296E3003178D0001308F000A122D
:1022D0000313C9230A167729733003178D000130C1
:1022E0008F000A120313C9230A16772977290C30A5
:1022F000CA000130CB000A127A230A160A128A1584
:1023000080260A168A117808B600360B88298C298F
:102310003608023C031DCA29B81C9029B901992925
:10232000370CF700F70C3F30F70577080739013E07
:10233000B900360BA129B90A3908093C0319B901BA
:10234000AC293608023C031DAC29B908031DAB2992
:102350000830B900AC29B903B908031DB129B81474
:10236000BF29B810B903390DF700F70DFC30F70598
:1023700077081C39B900E330B7053908B7040B30CA
:10238000BA003708BB0097201930BA003808BB00E4
:102390009720D1293608BA000A128A15D0260A16C3
:1023A0008A110A128A156E270A168A118A150A16C8
:1023B000362F0A1286270A164D30CD000A12B32393
:1023C0000A163030CD000A12B3230A162408BB00C7
:1023D0001830BC000A128A154A220A168A117A306D
:1023E00003178D0001308F0003140E300313BA0061
:1023F0000A128A15E8260A168A110A128A270A166C
:10240000250803190D2A013A0319172A033A03195B
:10241000212A013A03192B2A352A823003178D000D
:1024200001308F000A120313C9230A16362A873097
:1024300003178D0001308F000A120313C9230A16F7
:10244000362A8C3003178D0001308F000A120313D7
:10245000C9230A16362A913003178D0001308F00E8
:102460000A120313C9230A16362A362A0A128A15B3
:1024700080260A168A117808B600360B402A442AAC
:102480003608023C031D752A360B502A2508A50A7A
:10249000003A03194F2A2508043C0319A501572ABD
:1024A000A508031D562A0330A500572AA5030130AD
:1024B00003178D000313250803178C0083168C1354
:1024C0000C15831203130B08F7008B1383160317E5
:1024D00055308D00AA308D008C148C186D2A0C118B
:1024E0007708831203138B047C2A3608BA000A1279
:1024F0008A15D0260A168A110A128A156E270A161C
:102500008A118A150A16362F0A1286270A164D30A6
:10251000CD000A12B3230A163030CD000A12B323BD
:102520000A162408BB001830BC000A128A154A2279
:102530000A168A11983003178D0001308F0003149A
:102540000D300313BA000A128A15E8260A168A11FA
:102550000A128A270A1626080319BB2A013A031908
:10256000C52A033A0319CF2A013A0319D92A073A8F
:102570000319E32AED2AA03003178D0001308F00E4
:102580000A120313C9230A16EE2AA53003178D0079
:1025900001308F000A120313C9230A16EE2AAA304B
:1025A00003178D0001308F000A120313C9230A1686
:1025B000EE2AAF3003178D0001308F000A1203138B
:1025C000C9230A16EE2AB43003178D0001308F009C
:1025D0000A120313C9230A16EE2AEE2A0A128A15D2
:1025E00080260A168A117808B600360BF82AFC2ACB
:1025F0003608023C031D2D2B360B042BA60A260899
:10260000053C0319A6010F2B3608023C031D0F2BB6
:10261000A608031D0E2B0430A6000F2BA6030230C4
:1026200003178D000313260803178C0083168C13E1
:102630000C15831203130B08F7008B138316031773
:1026400055308D00AA308D008C148C18252B0C1160
:102650007708831203138B04342B3608BA000A124E
:102660008A15D0260A168A110A128A156E270A16AA
:102670008A118A150A16362F0A1286270A164D3035
:10268000CD000A12B3230A163030CD000A12B3234C
:102690000A162408BB001830BC000A128A154A2208
:1026A0000A168A11BB3003178D0001308F00031406
:1026B0000D300313BA000A128A15E8260A168A1189
:1026C0000A128A270A169030C3000E30C4000A127C
:1026D000AF240A167808B700371C782BC3300317CD
:1026E0008D0001308F000A120313C9230A16812BB3
:1026F000CC3003178D0001308F000A120313C92359
:102700000A160A128A1580260A168A117808B60057
:10271000360B8B2B8F2B3608023C031D9A2B371C54
:10272000932B3710942B37140E30BA003708BB00A8
:102730009720A12B3608BA000A128A15D0260A164D
:102740008A118A150A16362F0A1286270A164D3064
:10275000CD000A12B3230A163030CD000A12B3237B
:102760000A162408BB001830BC000A128A154A2237
:102770000A168A11D73003178D0001308F00031419
:102780000D300313BA000A128A15E8260A168A11B8
:102790000A128A270A169030C3000A30C4000A12AF
:1027A000AF240A167808B700DF3003178D00013018
:1027B0008F000A120313C9230A163708C0390319F8
:1027C000EB2B403A0319F62BC03A0319012C403A7F
:1027D00003190C2C172C3230CD000A12B3230A1621
:1027E0003430CD000A12B3230A16182C3230CD0033
:1027F0000A12B3230A163030CD000A12B3230A1688
:10280000182C3130CD000A12B3230A163630CD0011
:102810000A12B3230A16182C3330CD000A12B32340
:102820000A163230CD000A12B3230A16182C182CBF
:10283000E23003178D0001308F000A120313C92301
:102840000A160A128A1580260A168A117808B60016
:10285000360B2B2C2F2C3608023C031D482C370836
:10286000C039B8003F30B705360B382C4030B807B8
:102870003608023C031D3E2C4030B802C030B8057B
:102880003808B7040A30BA003708BB0097204F2C2D
:102890003608BA000A128A15D0260A168A118A1535
:1028A0000A16362F0A1286270A164D30CD000A1254
:1028B000B3230A163030CD000A12B3230A162408B7
:1028C000BB001830BC000A128A154A220A168A1167
:1028D000E93003178D0001308F0003140D3003130E
:1028E000BA000A128A15E8260A168A110A128A27DD
:1028F0000A169030C3000A30C4000A12AF240A1628
:102900007808B7003708303903198D2C103A0319AD
:10291000972C303A0319A12CAB2CF13003178D0002
:1029200001308F000A120313C9230A16AC2CFA30A7
:1029300003178D0001308F000A120313C9230A16F2
:10294000AC2C033003178D0002308F000A120313E2
:10295000C9230A16AC2CAC2C0A128A1580260A163A
:102960008A117808B600360BB62CBA2C3608023C11
:10297000031DDD2C37083039B800CF30B705360BD2
:10298000C72C1030B8073808303C0319B801360896
:10299000023C031DD32CB808031DD12C2030B800F5
:1029A000D32C1030B8023030B8053808B7040A30DC
:1029B000BA003708BB009720E42C3608BA000A1288
:1029C0008A15D0260A168A118A150A16362F0A1277
:1029D00086270A164D30CD000A12B3230A1630306E
:1029E000CD000A12B3230A162408BB001830BC001D
:1029F0000A128A154A220A168A110E3003178D0010
:102A000002308F0003140D300313BA000A128A1526
:102A1000E8260A168A110A128A270A169030C3007D
:102A20000D30C4000A12AF240A167808B700B708A0
:102A30000319242D163003178D0002308F000A125F
:102A40000313C9230A162D2D1F3003178D000230E2
:102A50008F000A120313C9230A160A128A15802648
:102A60000A168A117808B600360B372D3B2D36082A
:102A7000023C031D482DB7080319402DB701422D14
:102A8000FF30B7000D30BA003708BB0097204F2D3C
:102A90003608BA000A128A15D0260A168A118A1533
:102AA0000A16362F0A1286270A164D30CD000A1252
:102AB000B3230A162408BB001130BC000A128A1581
:102AC0004A220A168A112A3003178D0002308F001D
:102AD00003100E300313BA000A128A15E8260A16EC
:102AE0008A110A128A270A169030C3001330C400D4
:102AF0000A12AF240A167808B700B708031D8A2DFA
:102B0000323003178D0002308F000A120313C923DD
:102B10000A16932D3B3003178D0002308F000A12E6
:102B20000313C9230A160A128A1580260A168A1167
:102B30007808B600360B9D2DA12D3608023C031DEA
:102B4000AE2DB7080319A62DB701A82DFF30B70089
:102B50001330BA003708BB009720B52D3608BA00ED
:102B60000A128A15D0260A168A118A150A16362FD5
:102B70000A1286270A164D30CD000A12B3230A1610
:102B80002408BB001130BC000A128A154A220A161A
:102B90008A11463003178D0002308F0003100C306D
:102BA0000313BA000A128A15E8260A168A110A12B5
:102BB0008A270A169030C3000E30C4000A12AF24D0
:102BC0000A167808B700370806390319F12D023ABA
:102BD0000319FB2D063A0319052E023A03190F2E8D
:102BE000192E4D3003178D0002308F000A12031387
:102BF000C9230A161A2E563003178D0002308F0093
:102C00000A120313C9230A161A2E5F3003178D0008
:102C100002308F000A120313C9230A161A2E6830D5
:102C200003178D0002308F000A120313C9230A16FE
:102C30001A2E1A2E0A128A1580260A168A11780868
:102C4000B600360B242E282E3608023C031D472ED4
:102C50003608023C031D352E37080639031D332E76
:102C60000630B704352E0230B702360B412E370836
:102C70000639063C031D3F2EF930B705412E0230C0
:102C8000B7070E30BA003708BB0097204E2E360823
:102C9000BA000A128A15D0260A168A118A150A164F
:102CA000362F0A1286270A164D30CD000A12B3239A
:102CB0000A162408BB001130BC000A128A154A22E9
:102CC0000A168A11733003178D0002308F0003102B
:102CD0000D300313BA000A128A15E8260A168A1163
:102CE0000A128A270A169030C3001130C4000A1253
:102CF000AF240A167808B7009230C3001130C40020
:102D00000A12AF240A167808B800371F912E7A30BD
:102D100003178D0002308F000A120313C9230A160D
:102D20009A2E833003178D0002308F000A1203138E
:102D3000C9230A160A128A1580260A168A117808EB
:102D4000B600360BA42EA82E3608023C031DDF2E3B
:102D5000371FAD2E37133813AF2E37173817903073
:102D6000C5001130C6003708C7000A126A240A16C7
:102D70009230C5001130C6003808C7000A126A2414
:102D80000A16113003178D000313370803178C0040
:102D900083168C130C15831203130B08F7008B1387
:102DA0008316031755308D00AA308D008C148C18B3
:102DB000D72E0C117708831203138B04E62E3608E6
:102DC000BA000A128A15D0260A168A118A150A161E
:102DD000362F0A1286270A164D30CD000A12B32369
:102DE0000A162408BB001130BC000A128A154A22B8
:102DF0000A168A118E3003178D0002308F000310DF
:102E00000D300313BA000A128A15E8260A168A1131
:102E10000A128A270A169030C3001930C4000A1219
:102E2000AF240A167808B7009230C3001930C400E6
:102E30000A12AF240A167808B800371C292F9530DB
:102E400003178D0002308F000A120313C9230A16DC
:102E5000322F9E3003178D0002308F000A120313A9
:102E6000C9230A160A128A1580260A168A117808BA
:102E7000B600360B3C2F402F3608023C031D772F3F
:102E8000371C452F37103810472F3714381490301F
:102E9000C5001930C6003708C7000A126A240A168E
:102EA0009230C5001930C6003808C7000A126A24DB
:102EB0000A16193003178D000313370803178C0007
:102EC00083168C130C15831203130B08F7008B1356
:102ED0008316031755308D00AA308D008C148C1882
:102EE0006F2F0C117708831203138B047E2F360883
:102EF000BA000A128A15D0260A168A118A150A16ED
:102F0000362F0A1286270A164D30CD000A12B32337
:102F10000A162408BB001130BC000A128A154A2286
:102F20000A168A11A93003178D0002308F00031092
:102F30000D300313BA000A128A15E8260A168A1100
:102F40000A128A270A169030C3000A30C4000A12F7
:102F5000AF240A167808B700371DB82FB030031712
:102F60008D0002308F000A120313C9230A16C12FE5
:102F7000B53003178D0002308F000A120313C923E6
:102F80000A160A128A1580260A168A117808B600CF
:102F9000360BCB2FCF2F3608023C031DDA2F371DFF
:102FA000D32F3711D42F37150A30BA003708BB009A
:102FB0009720E12F3608BA000A128A15D0260A1681
:102FC0008A110A128A156E270A168A118A150A169C
:022FD000362F9A
:103000000A128A1186270A168A154D30CD000A1237
:103010008A11B3230A168A152408BB001130BC009C
:103020000A124A220A16BC3003178D0002308F00A4
:1030300003100D300313BA000A12E8260A160A120A
:103040008A118A270A168A159030C3000F30C400EF
:103050000A128A11AF240A168A157808B7000330BD
:10306000B705370803193E28013A03194A28033ADD
:1030700003195628013A031962286E28C330031732
:103080008D0002308F000A128A110313C9230A1619
:103090008A156F28CC3003178D0002308F000A127A
:1030A0008A110313C9230A168A156F28D53003170E
:1030B0008D0002308F000A128A110313C9230A16E9
:1030C0008A156F28DE3003178D0002308F000A1238
:1030D0008A110313C9230A168A156F286F280A124A
:1030E00080260A167808B600360B77287B28360823
:1030F000023C031DA8283608023C031D8628B70899
:10310000031D85280330B7008628B703360B8928AE
:10311000B70A3708043C0319B7013708FC3E031807
:10312000A028043EB028B801A0285530B800A02837
:10313000AA30B800A028FF30B800A028B801A02805
:103140000F30BA003808BB008A1197208A15AD28C5
:103150003608BA000A12D0260A168A150A16362F21
:103160000A108A100A1182079328952898289B280C
:10317000E830C3000330C4000A128A11AF240A16D3
:103180008A157808C0004013E830C5000330C60037
:103190004008C7000A128A116A240A168A15D02824
:1031A000D12800004017E830C5000330C6004008B1
:1031B000C7000A128A116A240A168A150230CB0047
:1031C0000A128A1102230A168A1508003A082F02E9
:1031D0000319D4293A08AF00E830C3000630C40010
:1031E0000A128A11AF240A168A157808BC00F0303A
:1031F000BC05E830C3000730C4000A128A11AF24AE
:103200000A168A157808BD00F330BD05E830C30002
:103210000230C4000A128A11AF240A168A157808EF
:10322000BE00F030BE05E830C3000330C4000A120F
:103230008A11AF240A168A157808BF00F330BF053B
:103240003A08013A03194F29033A03195329013A5D
:1032500003195829073A03195E29013A0319642909
:10326000033A03196A29013A03196F290F3A03191E
:103270007429013A03197929033A03197F29013A7C
:1032800003198429073A03198929013A03198E2958
:10329000033A03199429013A03199A299F29BE1464
:1032A0003D15BF15A0290930BC043D15BF15A02947
:1032B0000330BC04BE153D15BF15A0290530BC0464
:1032C000BE143D15BF15A0293C140630BE043D15A3
:1032D000BF15A0293C14BE14BD153F15A02905300B
:1032E000BC04BE14BD15A0293C140630BE04BD1597
:1032F000A0293C140630BE040C30BD04A0290530C2
:10330000BC04BE143F15A0293C140630BE043F1572
:10331000A0293C140630BE043D15A0290530BC048C
:10332000BE140C30BF04A0293C140630BE040C307F
:10333000BF04A0290530BC043D15BF15A029A02954
:10334000E830C5000230C6003E08C7000A128A11E4
:103350006A240A168A15E830C5000330C6003F0803
:10336000C7000A128A116A240A168A15E830C500B5
:103370000630C6003C08C7000A128A116A240A16E1
:103380008A15E830C5000730C6003D08C7000A129C
:103390008A116A240A168A153A08003C0318D429AF
:1033A0003A080F3C0318B82008003A082E02031907
:1033B0002D2A3A08AE00E830C3000630C4000A12D5
:1033C0008A11AF240A168A157808BC00CF30BC05D4
:1033D000E830C3000230C4000A128A11AF240A1672
:1033E0008A157808BE00CF30BE053A080319052AB1
:1033F000013A0319082A033A03190A2A013A031960
:103400000D2A073A0319102A122ABC163E16132A4F
:103410003E16132A3C16BE16132A3030BC04132A5B
:103420003C16132A132AE830C5000230C6003E08B5
:10343000C7000A128A116A240A168A15E830C500E4
:103440000630C6003C08C7000A128A116A240A1610
:103450008A153A08043C0318B8200800B608031976
:10346000992A250803193E2A013A03194B2A033ADF
:1034700003196A2A013A0319892A972ABA010A12FA
:103480008A1148260A168A153608BA00E620260848
:10349000BA00D521982A2208033C031C5D2A36086D
:1034A000BA00E6202608BA00D5210130BA000A1277
:1034B0008A1148260A168A15692ABA010A128A113F
:1034C00048260A168A153608BA00E6202608BA00E9
:1034D000D521982A2208033C03187C2A3608BA0012
:1034E000E6202608BA00D5210130BA000A128A1156
:1034F00048260A168A15882ABA010A128A1148260D
:103500000A168A153608BA00E6202608BA00D52120
:10351000982A2608BA00D5213608BA00E6200130DC
:10352000BA000A128A1148260A168A15982A982A79
:10353000A52ABA010A128A1148260A168A150F30DE
:10354000BA00E6200530BA00D5218A150A164E2F9A
:10355000A2010618AD2A0130A2078618B12A02304E
:10356000A2070619B52A0430A2073008220203195F
:10357000882B22080319D22A013A0319D22A033AC6
:103580000319D22A013A0319D22A073A0319F22A57
:10359000013A0319232B033A0319532B013A031958
:1035A0006C2B852BBB010A128A118F270A168A15EC
:1035B000EA30C5000330C600BD30C7000A128A11C8
:1035C0006A240A168A152208BB000A128A112D25C0
:1035D0000A168A150130BB000A128A11A4270A169E
:1035E0008A15862B9030C3000A30C4000A128A1153
:1035F000AF240A168A157808BA000F30BA05C03011
:10360000BA040A30C3003A08C4000A128A116F26AD
:103610000A168A150130BB000A128A118F270A1672
:103620008A15EA30C5000330C6007730C7000A1299
:103630008A116A240A168A15BB010A128A11A42764
:103640000A168A15862B9030C3000A30C4000A126D
:103650008A11AF240A168A157808BA000F30BA0505
:10366000BA160A30C3003A08C4000A128A116F263B
:103670000A168A150130BB000A128A118F270A1612
:103680008A15EA30C5000330C6007730C7000A1239
:103690008A116A240A168A15BB010A128A11A42704
:1036A0000A168A15862B0130BB000A128A118F2751
:1036B0000A168A15BB010A128A11A4270A168A154E
:1036C000EA30C5000330C600EE30C7000A128A1186
:1036D0006A240A168A15862B0130BB000A128A1149
:1036E0008F270A168A15BB010A128A11A4270A1607
:1036F0008A15EA30C5000330C600DB30C7000A1265
:103700008A116A240A168A15862B862B2208B00095
:103710009030C3000E30C4000A128A11AF240A167A
:103720008A157808B800B700861D982B3714992B96
:103730003710380837020319A62B0E30C30037089C
:10374000C4000A128A116F260A168A15EA30C300CD
:10375000C4010A128A11AF240A168A157808B90022
:10376000B91FB42BA601B62B0430A600391FBB2B02
:103770000330A500BC2BA50139082039031DCA2B35
:103780001930C3000230C4000A128A116F260A16CB
:103790008A15DB2B1930C300C4010A128A116F2667
:1037A0000A168A150B30C3008530C4000A128A112C
:1037B0006F260A168A150A128A1186270A168A1592
:1037C00022080319F92B013A0319052C033A0319AE
:1037D000112C013A03191D2C073A0319292C013A1F
:1037E0000319352C033A0319412C013A03194D2CC6
:1037F000592CC93003178D0000308F000A128A112E
:103800000313C9230A168A155A2CCE3003178D00CC
:1038100000308F000A128A110313C9230A168A1571
:103820005A2CD33003178D0000308F000A128A11F2
:103830000313C9230A168A155A2CD83003178D0092
:1038400000308F000A128A110313C9230A168A1541
:103850005A2CDD3003178D0000308F000A128A11B8
:103860000313C9230A168A155A2CE23003178D0058
:1038700000308F000A128A110313C9230A168A1511
:103880005A2CE73003178D0000308F000A128A117E
:103890000313C9230A168A155A2CEC3003178D001E
:1038A00000308F000A128A110313C9230A168A15E1
:1038B0005A2C5A2C0A1200200A167908BB007808E4
:1038C000BA007908BD007808BC000A128A117E2669
:1038D0000A168A150830CA00CB010A128A117A2307
:1038E0000A168A150A12BB220A160A128A118A2798
:1038F0000A168A152208053C031C822C0A1286240B
:103900000A16852C0A126B250A160A123D260A167B
:103910000A121D230A167808B900A508031D972C62
:10392000BA010A128A1148260A168A15AE2CB9085D
:103930000319A82C2608BA00D5213908BA00E620B8
:103940000130BA000A128A1148260A168A15AE2CCE
:10395000BA010A128A1148260A168A158A150A1609
:10396000502F840183131F308305FF30A0000130E6
:10397000A700A800A900AA00AC01AB01AD00AE01F0
:10398000AF010830B000831603170908C039890059
:1039900003131F129F120030031788008312870140
:1039A00088018901FF308316031385008600870094
:1039B0008312851083168510831205158316051151
:1039C0008312A201A501A6010230B600FA30CB0095
:1039D0000A128A1102230A168A15B60BE62C0A125D
:1039E0008A114B2D0A168A150A128A11D72D0A162A
:1039F0008A150A128A113B2E0A168A15BA010A1272
:103A00008A1148260A168A1587110530CB000A123A
:103A10008A1102230A168A15BD01BC010A128A11F5
:103A20007E260A168A15EA30C300C4010A128A11DA
:103A3000AF240A168A157808B2000A128A1186275E
:103A40000A168A15E73003178D0002308F000A121C
:103A50008A110313C9230A168A15321E412D0A1230
:103A60008A118A270A168A15F03003178D00023052
:103A70008F000A128A110313C9230A168A15B3018B
:103A8000532D0A128A118A270A168A15F93003174C
:103A90008D0002308F000A128A110313C9230A16FF
:103AA0008A150130B300C830CB000A128A110223F4
:103AB0000A168A150A1200200A167908B700780833
:103AC000B6007908BD007808BC000A128A117E266B
:103AD0000A168A150A1296280A160230B600FA301B
:103AE000CB000A128A1102230A168A15B60B6F2D13
:103AF000B3080319912D9030C5001130C6001D3058
:103B0000C7000A128A116A240A168A159230C50063
:103B10001130C6009D30C7000A128A116A240A16A5
:103B20008A150F30A300A4010A12BB210A16B501A1
:103B3000B401B308031D4F2F24080319CD2D013AFA
:103B40000319F72E033A0319FD2E013A0319032F27
:103B5000073A0319072F013A03190B2F033A0319E8
:103B60000F2F013A0319132F0F3A0319172F013A98
:103B700003191B2F033A03191F2F013A0319232F8F
:103B8000073A0319272F013A03192B2F033A031978
:103B90002F2F013A0319332F352F0A128A11862746
:103BA0000A168A1522080319F42D013A0319002E6A
:103BB000033A03190C2E013A0319182E073A031978
:103BC000242E013A0319302E033A03193C2E013AF0
:103BD0000319482E0F3A0319542E013A0319602E87
:103BE000033A03196C2E782EF13003178D00003044
:103BF0008F000A128A110313C9230A168A15842E0C
:103C0000F63003178D0000308F000A128A1103135B
:103C1000C9230A168A15842EFB3003178D00003045
:103C20008F000A128A110313C9230A168A15842EDB
:103C3000003003178D0001308F000A128A11031320
:103C4000C9230A168A15842E053003178D0001300A
:103C50008F000A128A110313C9230A168A15842EAB
:103C60000A3003178D0001308F000A128A110313E6
:103C7000C9230A168A15842E0F3003178D000130D0
:103C80008F000A128A110313C9230A168A15842E7B
:103C9000143003178D0001308F000A128A110313AC
:103CA000C9230A168A15842E193003178D00013096
:103CB0008F000A128A110313C9230A168A15842E4B
:103CC0001E3003178D0001308F000A128A11031372
:103CD000C9230A168A15842E233003178D0001305C
:103CE0008F000A128A110313C9230A168A15842E1B
:103CF000283003178D0001308F000A128A11031338
:103D0000C9230A168A15842E0A1200200A16790879
:103D1000BA007808B9007908BD007808BC000A121A
:103D20008A117E260A168A150830CA00CB010A12AB
:103D30008A117A230A168A150A12BB220A160A1257
:103D40008A118A270A168A152208043C0318AC2E09
:103D50002208063C0318B02E0A1286240A16B32E37
:103D60000A126B250A160A123D260A160A12802626
:103D70000A167808B600360BBE2EC22E3608023C54
:103D8000031DF12E360BCA2EA20A22080B3C031982
:103D9000A201D12EA208031DD02E0A30A200D12EDE
:103DA000A2030A12BB210A1603178D01031322086E
:103DB00003178C0083168C130C15831203130B0846
:103DC000F7008B138316031755308D00AA308D0032
:103DD0008C148C18E92E0C117708831203138B04B2
:103DE000F62E3608BA000A12D0260A16362F0130EF
:103DF000B6008A1100208A15362F0230B6008A11CB
:103E000000208A15362F8A11C7288A15362F8A1165
:103E1000D9298A15362F8A11842A8A15362F8A11B4
:103E20003C2B8A15362F8A11A42B8A15362F8A111E
:103E3000522C8A15362F8A11E72C8A15362F8A11B3
:103E4000522D8A15362F8A11B82D8A15362F8A11D0
:103E5000512E8A15362F8A11E92E8A15362F8A118E
:103E6000812F8A15362F0028362F362F0A12002070
:103E70000A167908B7007808B6007908BD007808F6
:103E8000BC000A128A117E260A168A150A121D2300
:103E90000A167808B1003108B6002E2A502FA82A39
:103EA0003408323C031D592FB508031D592F8514C2
:0C3EB0005C2FB40A0319B50A992D6300B9
:04400E00822CFF3FC2
:00000001FF
